 SwiQdl

 Timestamp is 54865970 (Tue Dec 09 10:07:44 2014)

 Preferred load address is 10000000

 Start         Length     Name                   Class
 0001:00000000 000070dcH .text                   CODE
 0002:00000000 000040b8H .rdata                  DATA
 0002:000040b8 0000006fH .rdata$debug            DATA
 0002:00004128 00000014H .xdata                  DATA
 0002:0000413c 00000014H .idata$2                DATA
 0002:00004150 00000014H .idata$3                DATA
 0002:00004164 0000009cH .idata$4                DATA
 0002:00004200 0000001eH .idata$6                DATA
 0002:00004220 0000006aH .edata                  DATA
 0003:00000000 0000009cH .idata$5                DATA
 0003:0000009c 00000004H .CRT$XCA                DATA
 0003:000000a0 00000004H .CRT$XCAA               DATA
 0003:000000a4 00000004H .CRT$XCZ                DATA
 0003:000000a8 00000004H .CRT$XIA                DATA
 0003:000000ac 00000004H .CRT$XIZ                DATA
 0003:000000b0 00000004H .CRT$XPA                DATA
 0003:000000b4 00000004H .CRT$XPZ                DATA
 0003:000000b8 00000004H .CRT$XTA                DATA
 0003:000000bc 00000004H .CRT$XTZ                DATA
 0003:000000c0 00000654H .data                   DATA
 0003:00000718 00000364H .bss                    DATA
 0004:00000000 00000150H .pdata                  DATA
 0005:00000000 00000058H .rsrc$01                DATA
 0005:00000060 00000408H .rsrc$02                DATA

  Address         Publics by Value              Rva+Base       Lib:Object

 0000:00000000       ___safe_se_handler_count   00000000     <absolute>
 0000:00000000       ___safe_se_handler_table   00000000     <absolute>
 0001:00000000       CalculateCRC16             10001000 f   crc.obj
 0001:00000094       ?DisplayMemoryStatus@@YAXXZ 10001094 f   swiusb.obj
 0001:000000f4       ?OpenOutModemBulkPipe11@@YAPAXU_USB_ENDPOINT_DESCRIPTOR@@@Z 100010f4 f   swiusb.obj
 0001:000001dc       ?OpenInModemBulkPipe10@@YAPAXU_USB_ENDPOINT_DESCRIPTOR@@@Z 100011dc f   swiusb.obj
 0001:000002c4       ?GetChannel@@YAPAU_SW_CHANNEL@@PAU1@K@Z 100012c4 f   swiusb.obj
 0001:0000036c       ?dumpBytesData@@YAXKPA_WPAEK@Z 1000136c f   swiusb.obj
 0001:00000620       ?SWIReadCompletionRoutine@@YAKPAX@Z 10001620 f   swiusb.obj
 0001:0000065c       ?SWIWriteCompletionRoutine@@YAKPAX@Z 1000165c f   swiusb.obj
 0001:000006a0       ?BulkInThread@@YAXPAPAX@Z  100016a0 f   swiusb.obj
 0001:00001154       ?BulkOutThread@@YAXPAPAX@Z 10002154 f   swiusb.obj
 0001:00001b60       ?USBDeviceNotifications@@YAHPAXKPAPAK111@Z 10002b60 f   swiusb.obj
 0001:00002a18       USBDeviceAttach            10003a18 f   swiusb.obj
 0001:0000436c       USBInstallDriver           1000536c f   swiusb.obj
 0001:000043c4       ?VerifyPacket@@YAHPAEK@Z   100053c4 f   swiusb.obj
 0001:00004518       ?HandleErrorResponse@@YAXXZ 10005518 f   swiusb.obj
 0001:00004648       ?ProcessPacket@@YAXPAU_SW_CHANNEL@@PAEI@Z 10005648 f   swiusb.obj
 0001:00004d80       ?SendData@@YAHPAU_SW_CHANNEL@@@Z 10005d80 f   swiusb.obj
 0001:000053a0       ?ValidateData@@YAKPAU_SW_CHANNEL@@PAXK@Z 100063a0 f   swiusb.obj
 0001:000055e4       ?BuildPacket@@YAHPAU_SW_CHANNEL@@@Z 100065e4 f   swiusb.obj
 0001:00005ca4       ?StateMachineThread@@YAKPAX@Z 10006ca4 f   swiusb.obj
 0001:00005ff4       ?GetFWFile@@YAHAAU_GOBI_FW@@@Z 10006ff4 f   swiusb.obj
 0001:00006238       ?GetGobiFirmware@@YAHXZ    10007238 f   swiusb.obj
 0001:00006970       SetEvent                   10007970 f i swiusb.obj
 0001:000069a4       ResetEvent                 100079a4 f i swiusb.obj
 0001:000069d8       GetCurrentThreadId         100079d8 f i swiusb.obj
 0001:000069f8       RemoveTailList             100079f8 f i swiusb.obj
 0001:00006a68       NKDbgPrintfW               10007a68 f   coredll:COREDLL.dll
 0001:00006a78       GlobalMemoryStatus         10007a78 f   coredll:COREDLL.dll
 0001:00006a88       GetLastError               10007a88 f   coredll:COREDLL.dll
 0001:00006a98       memcpy                     10007a98 f   coredll:COREDLL.dll
 0001:00006aa8       wcscat                     10007aa8 f   coredll:COREDLL.dll
 0001:00006ab8       wsprintfW                  10007ab8 f   coredll:COREDLL.dll
 0001:00006ac8       rand                       10007ac8 f   coredll:COREDLL.dll
 0001:00006ad8       EventModify                10007ad8 f   coredll:COREDLL.dll
 0001:00006ae8       GetTickCount               10007ae8 f   coredll:COREDLL.dll
 0001:00006af8       VirtualFree                10007af8 f   coredll:COREDLL.dll
 0001:00006b08       Sleep                      10007b08 f   coredll:COREDLL.dll
 0001:00006b18       WaitForMultipleObjects     10007b18 f   coredll:COREDLL.dll
 0001:00006b28       WaitForSingleObject        10007b28 f   coredll:COREDLL.dll
 0001:00006b38       VirtualAlloc               10007b38 f   coredll:COREDLL.dll
 0001:00006b48       swprintf                   10007b48 f   coredll:COREDLL.dll
 0001:00006b58       __rt_udiv                  10007b58 f   coredll:COREDLL.dll
 0001:00006b68       LocalFree                  10007b68 f   coredll:COREDLL.dll
 0001:00006b78       TerminateThread            10007b78 f   coredll:COREDLL.dll
 0001:00006b88       CloseHandle                10007b88 f   coredll:COREDLL.dll
 0001:00006b98       CeSetThreadPriority        10007b98 f   coredll:COREDLL.dll
 0001:00006ba8       CreateThread               10007ba8 f   coredll:COREDLL.dll
 0001:00006bb8       LocalAllocTrace            10007bb8 f   coredll:COREDLL.dll
 0001:00006bc8       memset                     10007bc8 f   coredll:COREDLL.dll
 0001:00006bd8       CreateEventW               10007bd8 f   coredll:COREDLL.dll
 0001:00006be8       RegCloseKey                10007be8 f   coredll:COREDLL.dll
 0001:00006bf8       RegQueryValueExW           10007bf8 f   coredll:COREDLL.dll
 0001:00006c08       RegOpenKeyExW              10007c08 f   coredll:COREDLL.dll
 0001:00006c18       MultiByteToWideChar        10007c18 f   coredll:COREDLL.dll
 0001:00006c28       ReadFile                   10007c28 f   coredll:COREDLL.dll
 0001:00006c38       SetFilePointer             10007c38 f   coredll:COREDLL.dll
 0001:00006c48       strcpy                     10007c48 f   coredll:COREDLL.dll
 0001:00006c58       GetFileSize                10007c58 f   coredll:COREDLL.dll
 0001:00006c68       CreateFileW                10007c68 f   coredll:COREDLL.dll
 0001:00006c78       wcscmp                     10007c78 f   coredll:COREDLL.dll
 0001:00006c88       _wcslwr                    10007c88 f   coredll:COREDLL.dll
 0001:00006c98       _DllMainCRTStartup         10007c98 f   corelibc:pegdmain.obj
 0001:00006d30       __security_check_cookie    10007d30     corelibc:armsecgs.obj
 0001:00006d44       __gsfailure                10007d44     corelibc:armsecgs.obj
 0001:00006d88       GetCurrentProcess          10007d88 f i corelibc:crt0dat.obj
 0001:00006dc4       _cinit                     10007dc4 f   corelibc:crt0dat.obj
 0001:00006f34       exit                       10007f34 f   corelibc:crt0dat.obj
 0001:00006f4c       _exit                      10007f4c f   corelibc:crt0dat.obj
 0001:00006f64       _cexit                     10007f64 f   corelibc:crt0dat.obj
 0001:00006f80       _c_exit                    10007f80 f   corelibc:crt0dat.obj
 0001:00006fcc       DllMain                    10007fcc f   corelibc:dllmain.obj
 0001:00006fe4       __security_init_cookie     10007fe4 f   corelibc:seccinit.obj
 0001:00007034       __GSHandlerCheckCommon     10008034 f   LIBCMTD:gshandler.obj
 0001:0000707c       __GSHandlerCheck           1000807c f   LIBCMTD:gshandler.obj
 0001:000070ac       __report_gsfailure         100080ac f   coredll:COREDLL.dll
 0001:000070bc       DisableThreadLibraryCalls  100080bc f   coredll:COREDLL.dll
 0001:000070cc       __security_gen_cookie      100080cc f   coredll:COREDLL.dll
 0002:0000413c       __IMPORT_DESCRIPTOR_COREDLL 1000d13c     coredll:COREDLL.dll
 0002:00004150       __NULL_IMPORT_DESCRIPTOR   1000d150     coredll:COREDLL.dll
 0003:00000000       __imp_NKDbgPrintfW         1000e000     coredll:COREDLL.dll
 0003:00000004       __imp_GlobalMemoryStatus   1000e004     coredll:COREDLL.dll
 0003:00000008       __imp_GetLastError         1000e008     coredll:COREDLL.dll
 0003:0000000c       __imp_memcpy               1000e00c     coredll:COREDLL.dll
 0003:00000010       __imp_wcscat               1000e010     coredll:COREDLL.dll
 0003:00000014       __imp_wsprintfW            1000e014     coredll:COREDLL.dll
 0003:00000018       __imp_rand                 1000e018     coredll:COREDLL.dll
 0003:0000001c       __imp_EventModify          1000e01c     coredll:COREDLL.dll
 0003:00000020       __imp_GetTickCount         1000e020     coredll:COREDLL.dll
 0003:00000024       __imp_VirtualFree          1000e024     coredll:COREDLL.dll
 0003:00000028       __imp_Sleep                1000e028     coredll:COREDLL.dll
 0003:0000002c       __imp_WaitForMultipleObjects 1000e02c     coredll:COREDLL.dll
 0003:00000030       __imp_WaitForSingleObject  1000e030     coredll:COREDLL.dll
 0003:00000034       __imp_VirtualAlloc         1000e034     coredll:COREDLL.dll
 0003:00000038       __imp_swprintf             1000e038     coredll:COREDLL.dll
 0003:0000003c       __imp___rt_udiv            1000e03c     coredll:COREDLL.dll
 0003:00000040       __imp_LocalFree            1000e040     coredll:COREDLL.dll
 0003:00000044       __imp_TerminateThread      1000e044     coredll:COREDLL.dll
 0003:00000048       __imp_CloseHandle          1000e048     coredll:COREDLL.dll
 0003:0000004c       __imp_CeSetThreadPriority  1000e04c     coredll:COREDLL.dll
 0003:00000050       __imp_CreateThread         1000e050     coredll:COREDLL.dll
 0003:00000054       __imp_LocalAllocTrace      1000e054     coredll:COREDLL.dll
 0003:00000058       __imp_memset               1000e058     coredll:COREDLL.dll
 0003:0000005c       __imp_CreateEventW         1000e05c     coredll:COREDLL.dll
 0003:00000060       __imp_RegCloseKey          1000e060     coredll:COREDLL.dll
 0003:00000064       __imp_RegQueryValueExW     1000e064     coredll:COREDLL.dll
 0003:00000068       __imp_RegOpenKeyExW        1000e068     coredll:COREDLL.dll
 0003:0000006c       __imp_MultiByteToWideChar  1000e06c     coredll:COREDLL.dll
 0003:00000070       __imp_ReadFile             1000e070     coredll:COREDLL.dll
 0003:00000074       __imp_SetFilePointer       1000e074     coredll:COREDLL.dll
 0003:00000078       __imp_strcpy               1000e078     coredll:COREDLL.dll
 0003:0000007c       __imp_GetFileSize          1000e07c     coredll:COREDLL.dll
 0003:00000080       __imp_CreateFileW          1000e080     coredll:COREDLL.dll
 0003:00000084       __imp_wcscmp               1000e084     coredll:COREDLL.dll
 0003:00000088       __imp__wcslwr              1000e088     coredll:COREDLL.dll
 0003:0000008c       __imp___report_gsfailure   1000e08c     coredll:COREDLL.dll
 0003:00000090       __imp_DisableThreadLibraryCalls 1000e090     coredll:COREDLL.dll
 0003:00000094       __imp___security_gen_cookie 1000e094     coredll:COREDLL.dll
 0003:00000098       \177COREDLL_NULL_THUNK_DATA 1000e098     coredll:COREDLL.dll
 0003:0000009c       __xc_a                     1000e09c     corelibc:crt0init.obj
 0003:000000a4       __xc_z                     1000e0a4     corelibc:crt0init.obj
 0003:000000a8       __xi_a                     1000e0a8     corelibc:crt0init.obj
 0003:000000ac       __xi_z                     1000e0ac     corelibc:crt0init.obj
 0003:000000b0       __xp_a                     1000e0b0     corelibc:crt0init.obj
 0003:000000b4       __xp_z                     1000e0b4     corelibc:crt0init.obj
 0003:000000b8       __xt_a                     1000e0b8     corelibc:crt0init.obj
 0003:000000bc       __xt_z                     1000e0bc     corelibc:crt0init.obj
 0003:000002c0       dpCurSettings              1000e2c0     swiusb.obj
 0003:00000704       ?fFWFolder@@3HA            1000e704     swiusb.obj
 0003:00000708       ?gdwMaxRetries@@3KA        1000e708     swiusb.obj
 0003:0000070c       __security_cookie_complement 1000e70c     corelibc:seccook.obj
 0003:00000710       __security_cookie          1000e710     corelibc:seccook.obj
 0003:00000718       ?ghDeviceInstalledEvent@@3PAXA 1000e718     swiusb.obj
 0003:0000071c       ?hDeviceCloseEvent@@3PAXA  1000e71c     swiusb.obj
 0003:00000720       ?hAbortEvent@@3PAXA        1000e720     swiusb.obj
 0003:00000724       ?ghQDLEvent@@3PAXA         1000e724     swiusb.obj
 0003:00000728       ?ghShutDownEvent@@3PAXA    1000e728     swiusb.obj
 0003:0000072c       ?ghShutDownRequestEvent@@3PAXA 1000e72c     swiusb.obj
 0003:00000730       ?gfGobi3k@@3HA             1000e730     swiusb.obj
 0003:00000734       ?gdwRetries@@3KA           1000e734     swiusb.obj
 0003:00000738       ?gModem@@3U_SW_MODEM@@A    1000e738     swiusb.obj
 0003:00000a6c       __onexitend                1000ea6c     <common>
 0003:00000a70       __onexitbegin              1000ea70     <common>
 0003:00000a74       _exitflag                  1000ea74     <common>
 0003:00000a78       _pRawDllMain               1000ea78     <common>

 entry point at        0001:00006c98

 Static symbols

 0001:00001510       ?TransmitBytes@@YAHPAU_SW_CHANNEL@@PAEI@Z 10002510 f   swiusb.obj
 0001:0000447c       ?ParseAndAddToReadQueue@@YAXPAEIPAU_SW_CHANNEL@@@Z 1000547c f   swiusb.obj
 0001:00006d90       _initterm                  10007d90 f   corelibc:crt0dat.obj
 0001:00006e30       doexit                     10007e30 f   corelibc:crt0dat.obj

 Exports

  ordinal    name

        1    USBDeviceAttach
        2    USBInstallDriver
